:0200000480007A
:100000006F00C0006F20802C6F20402C93000000F8
:10001000130100009301000013020000930200008E
:100020001303000093030000130400009304000076
:10003000130500009305000013060000930600005E
:100040001307000093070000130800009308000046
:100050001309000093090000130A0000930A00002E
:10006000130B0000930B0000130C0000930C000016
:10007000130D0000930D0000130E0000930E0000FE
:10008000130F0000930F000097020000938202F804
:100090007390523017B100001301C1E4F32240F114
:1000A0009392C2003301510073100134EF20900B82
:1000B000173500001305858B6F20006B8332851088
:1000C000739012148330850003310501833185015B
:1000D000033205028332850203330503833385032C
:1000E000033405048334850483358505033605060A
:1000F00083368506033705078337850703380508E8
:10010000833885080339050983398509033A050AC7
:10011000833A850A033B050B833B850B033C050CA7
:10012000833C850C033D050D833D850D033E050E87
:10013000833E850E033F050F833F850F033505057D
:10014000730020107311011423341100233C31007B
:10015000233041022334510223386102233C7102CF
:1001600023308104233491042338A104233CB104B7
:100170002330C1062334D1062338E106233CF1069F
:10018000233001092334110923382109233C310983
:100190002330410B2334510B2338610B233C710B6B
:1001A0002330810D2334910D2338A10D233CB10D53
:1001B0002330C10F2334D10F2338E10F233CF10F3B
:1001C000F312011423385100F32200102330511090
:1001D000F322101423345110F32230142338511019
:1001E000F3222014233C5110130501006F208033AB
:1010000000000000000000000000000000000000E0
:1010100000000000000000000000000000000000D0
:1010200000000000000000000000000000000000C0
:1010300000000000000000000000000000000000B0
:081040000000000000000000A8
:10200000B367B500B3E7C70093F77700B306C50021
:10201000638407023386C50093070500637ED502FB
:1020200003C705009385150093871700A38FE7FE6C
:10203000E398C5FE67800000E37ED5FE93070500A8
:1020400003B70500938787009385850023BCE7FECF
:10205000E3E8D7FE6780000067800000130101FFFE
:10206000B367C500233081002334110093F7770054
:10207000130405003307C500638207026376E50099
:1020800093F5F50FEFF09FFD8330810013050400F9
:1020900003340100130101016780000093F5F50F7F
:1020A00093968500B3E6B60093970601B3E7D70091
:1020B00093960702B3E6F600E378E5FC9307050084
:1020C0009387870023BCD7FEE3ECE7FE83308100D3
:1020D00013050400033401001301010167800000AF
:1020E00083470500638E07009307050003C71700A9
:1020F00093871700E31C07FE3385A7406780000025
:1021000013050000678000008347050093851500D4
:102110001305150003C7F5FF638A0700E386E7FE92
:102120001B8507003B05E5406780000013050000A4
:102130006FF05FFFB367B50093F77700639E070208
:10214000137886FF330805016378050393070500BC
:102150006F000001938787009385850063F807016E
:1021600083B6070003B70500E386E6FE3385A74084
:102170003306A640138507003386C5006F00400173
:1021800003C705008347F5FF93851500639AE700B1
:1021900013051500E396C5FE1305000067800000D7
:1021A0003B85E740678000009307050003C70500F3
:1021B0009387170093851500A38FE7FEE31807FEAA
:1021C000678000000347050093060002930705009F
:1021D0006318D70003C7170093871700E30CD7FED7
:1021E0009306D0026300D7069306B0026300D704BB
:1021F00083C60700930500006382060413050000F0
:1022000093871700131725001B8606FD83C607005A
:102210003307A700131717003305E600E39206FE05
:10222000638005023305A0406780000083C6170065
:102230009305000093871700E39206FC1305000046
:102240006780000083C6170093051000938717006E
:10225000E39606FA130500006FF09FFE8347050022
:10226000638007049305101017F7FFFF130787D942
:10227000939505030336070013051500B3E6B70071
:10228000630A060097F7FFFF23BE07DA83370700CC
:10229000E39A07FE2330D70083470500E39C07FC41
:1022A0006780000017F7FFFF1307C7D583370700C4
:1022B000638A070097F7FFFF23B607D88337070025
:1022C000E39A07FE2330A7006F000000130101FF0F
:1022D0001305903423341100EFF0DFFC130101FEED
:1022E0001306810093077101130890006F008000AE
:1022F000930707009376F500138706009305000304
:102300006374D800930570053B07B7002380E7008E
:10231000135545001387F7FFE31CF6FC8347810044
:10232000230C0100638207041305101093060600B6
:1023300017F7FFFF130707CD1315050383350700B4
:102340009386160033E6A700638A050097F7FFFF20
:1023500023BA07CE83370700E39A07FE83C7060038
:102360002330C700E39C07FC1301010267800000D3
:10237000130101FF37F8FFFF233411003307050174
:10238000B7E703006378F7141357C5009306076097
:1023900017460000130606C793973600B307F600EA
:1023A00083B70700337505016390070E978500001A
:1023B0009385C5C503B805006302081483378800F8
:1023C0009788000083B808C423B0F500638E170F08
:1023D0008337080093983600B308160193D7C700D7
:1023E0009397A70013E3F70D93E5F70123B0680077
:1023F00073000512973700009387C7C01317470073
:10240000B387E70003B7070063140710033708001A
:10241000B708040023B0E7000337880023B4E700BF
:10242000F3A80810B707E0FFB307F500371800005E
:10243000130705003388070103BF070083BE870029
:1024400003BE070103B387012330E7012334D7011B
:102450002338C701233C670093870702130707024D
:10246000E39C07FD7390081093973600B306F600BF
:1024700023B0B600730005120F10000083308100F6
:10248000130101016780000013F70704630A0702C4
:1024900013F70708631A07041307F00093E7070808
:1024A0006394E50493963600B306D60023B0F60095
:1024B0007300051283308100130101016780000061
:1024C00093E707046FF01FFE9787000023BC07B255
:1024D0006FF01FF0171500001305C592EFF01FD81D
:1024E00013053000EFF01FDC1715000013050596EB
:1024F000EFF0DFD613053000EFF0DFDA171500003C
:1025000013054599EFF09FD513053000EFF09FD9E3
:102510001715000013058599EFF05FD413053000FF
:10252000EFF05FD883358511130101F82338810658
:10253000233C11062334910623302107233C310527
:10254000233841052334510523306105233C7103B1
:1025500023388103233491032330A103233CB101A9
:102560009307800013040500638AF50E930720008B
:102570006380F506938745FF130710006376F70025
:102580009307F0006392F51A03350411EFF05FDE54
:102590001305040003340107833081078334810667
:1025A0000339010683398105033A0105833A810421
:1025B000033B0104833B8103033C0103833C810211
:1025C000033D0102833D8101130101086FD01FAF5C
:1025D000033785109377370063980706EF0780006D
:1025E000731030000327070083A70700630AF7046E
:1025F0001305101093071004971600009386068F9A
:1026000017F7FFFF130707A013150503833507000E
:102610009386160033E6A700638A050097F7FFFF4D
:1026200023B207A283370700E39A07FE83C7060099
:102630002330C700E39C07FC13053000EFF09FC672
:1026400013051000EFF01FC61715000013050594C1
:10265000EFF0DFC013053000EFF0DFC403290505FC
:10266000371C0000973400009384C499974B0000F6
:10267000938B4B99370B0400B70AE0FF978D00004E
:10268000938D4D98178A0000130A4A98B7F90300F2
:102690006F0080012334F70023B0FD00B71700005E
:1026A000330CFC00630E3C0B9357CC001394470093
:1026B0003387840003370700E30207FE9387076030
:1026C00093973700B387FB0083BC070093F70C0494
:1026D000638E0706732D0B1037160000B3055C01DF
:1026E00013050C002334B100EFF0DFA4630E0500E6
:1026F00093FC0C088335810063800C0437160000BE
:1027000013050C00EFF0DF8FB387840073100D10FA
:1027100003B70D0023B00700E31E07F623B0FD004A
:102720002330FA006FF09FF7171500001305858816
:10273000EFF0DFB26FF05FF0171500001305858131
:10274000EFF0DFB113053000EFF0DFB51705000043
:102750001305C57CEFF09FB013053000EFF09FB478
:1027600013050900EFF01FB4F32740F1639A07182F
:102770009767000093870789130101ED93D7C7007E
:1027800023308112177800001308C887130405004E
:102790009397A700175500001305C586233411121F
:1027A0009356C5001357C80093E7170097480000D9
:1027B000938848851306F0FF233CF5FE9396A60008
:1027C0001317A700B707002093E61600136717003A
:1027D00093D5C8001313F6039387F70C233CF8FE38
:1027E00023B0D8002330E500B3E7650073900718E5
:1027F00073270018639EE7141356B6009307F00181
:102800009702000093824201F39252307310063B0C
:102810007390073A739052301308F0BF13185801A1
:1028200097E7FFFF93874792B3870701739057108D
:10283000F3270034B387070173900714B7B700007C
:102840009B87071073902730B7E701009B870760CD
:10285000739007307350403017370000130787B963
:102860009307083EB3060701B307F700B70808004F
:1028700017760000233CD67817330000130383F645
:102880009776000023B0F6789388F8039307300317
:102890001308080113D61700B3861701B347F600D3
:1028A000B30507019396C600939757002330D700CE
:1028B0002334B70093F7070213070701B367F60045
:1028C000E31AE3FC13060012930500001305010050
:1028D0009737000023B407F0EFF04FF8B7070080F8
:1028E0003304F4001305010023348110EFD00FFDF1
:1028F0008330811203340112130101136780000039
:1029000013071000B7D7DB0A370608009387079133
:102910001306C6FF1315F7019316E7036F00C001F6
:102920002F20070013D71700B3C7E7009397E703DB
:10293000B3F7D700B3E7E70033F7C70093F5170005
:102940003307A700E39E05FC032007006FF09FFDFF
:102950001705000013050569EFF05F9013053000BF
:10296000EFF05F946780000097100000938080690B
:102970001301A00A23902000039700009303A00AEC
:1029800093012000631E77449710000093808067B6
:1029900037B1FFFF1B0101A0239120000397200006
:1029A000B7B3FFFF9B8303A093013000631A774204
:1029B00097100000938000653711EFBE1B0101AA3C
:1029C0002392200003A74000B713EFBE9B8303AA06
:1029D0009301400063167740971000009380806257
:1029E00037A1FFFF1B01A100239320000397600084
:1029F000B7A3FFFF9B83A300930150006312773EB0
:102A0000971000009380E0601301A00A239D20FE30
:102A10000397A0FF9303A00A930160006312773C21
:102A2000971000009380E05E37B1FFFF1B0101A00B
:102A3000239E20FE0397C0FFB7B3FFFF9B8303A035
:102A400093017000631E7738971000009380605CDC
:102A5000371100001B0101AA239F20FE0397E0FF0E
:102A6000B71300009B8303AA93018000631A773693
:102A7000971000009380E05937A1FFFF1B01A100D0
:102A80002390200003970000B7A3FFFF9B83A300C0
:102A9000930190006316773497100000938080575D
:102AA000375134121B018167138200FE231022026A
:102AB00083920000B75300009B8383679301A000BB
:102AC00063907232971000009380C0543731000039
:102AD0001B0181099380B0FFA3932000171200000F
:102AE0001302625383120200B73300009B838309F1
:102AF0009301B0006396722E9301C0001302000090
:102B0000B7D0FFFF9B80D0CD171100001301814F7C
:102B10002310110003170100B7D3FFFF9B83D3CD10
:102B20006310772C1302120093022000E31A52FC68
:102B30009301D00013020000B7C0FFFF9B80D0CCF0
:102B4000171100001301014C1300000023111100A4
:102B500003172100B7C3FFFF9B83D3CC63127728F1
:102B60001302120093022000E31852FC9301E000CC
:102B700013020000B7C0FFFF9B80C0BC171100000C
:102B8000130141481300000013000000231211003C
:102B900003174100B7C3FFFF9B83C3BC63127724B5
:102BA0001302120093022000E31652FC9301F0007E
:102BB00013020000B7B0FFFF9B80C0BB13000000F2
:102BC00017110000130101442313110003176100C2
:102BD000B7B3FFFF9B83C3BB6314772013021200BC
:102BE00093022000E31852FC93010001130200003D
:102BF000B7B0FFFF9B80B0AB1300000017110000BF
:102C00001301414013000000231411000317810039
:102C1000B7B3FFFF9B83B3AB6314771C130212009F
:102C200093022000E31652FC9301100113020000EE
:102C3000B7E0FFFF9B80B0AA130000001300000064
:102C4000171100001301013C231511000317A10007
:102C5000B7E3FFFF9B83B3AA631477181302120034
:102C600093022000E31652FC93012001130200009E
:102C70001711000013010139B72000009B80302399
:102C80002310110003170100B72300009B83332397
:102C9000631877141302120093022000E31A52FC07
:102CA0009301300113020000171100001301813558
:102CB000B71000009B803022130000002311110088
:102CC00003172100B71300009B833322631A771088
:102CD0001302120093022000E31852FC93014001FA
:102CE00013020000171100001301C131B7100000DA
:102CF0009B8020121300000013000000231211001B
:102D000003174100B71300009B832312631A770C4B
:102D10001302120093022000E31652FC93015001AB
:102D200013020000171100001301C12D1300000051
:102D30009300201123131100031761009303201146
:102D40006310770A1302120093022000E31C52FC66
:102D50009301600113020000171100001301812A82
:102D60001300000093001001130000002314110051
:102D700003178100930310016314770613021200F6
:102D800093022000E31A52FC930170011302000029
:102D900017110000130101271300000013000000A9
:102DA000B73000009B801000231511000317A1000D
:102DB000B73300009B8313006314770213021200E1
:102DC00093022000E31652FC37C500001B05F5EE08
:102DD00097150000938505232393A500631A3000FF
:102DE00013951100630005001365150073000000C2
:0C2DF0001305100073000000731000C0F9
:102E0000417373657274696F6E206661696C656485
:102E10003A2061646472203E3D202831554C203CAC
:102E20003C203132292026262061646472203C2017
:102E30003633202A202831554C203C3C2031322981
:102E40000A00000000000000417373657274696F2E
:102E50006E206661696C65643A20212870745B336A
:102E60005D5B616464722F2831554C203C3C2031FD
:102E700032295D202620307830383029202626203F
:102E80006361757365203D3D203078660A0000005F
:102E9000417373657274696F6E206661696C6564F5
:102EA0003A206E6F64650A00417373657274696FCE
:102EB0006E206661696C65643A20757365725F6D3A
:102EC000617070696E675B616464722F2831554C64
:102ED000203C3C203132295D2E61646472203D3DEE
:102EE00020300A0000000000417373657274696F3E
:102EF0006E206661696C65643A202122696C6C659C
:102F000067616C20696E737472756374696F6E2289
:102F10000A00000000000000417373657274696F5D
:102F20006E206661696C65643A2070745B335D5B2A
:102F3000616464722F2831554C203C3C2031322989
:102F40005D20262030783034300A00000000000078
:102F5000417373657274696F6E206661696C656434
:102F60003A2070745B335D5B616464722F28315565
:102F70004C203C3C203132295D20262030783038EE
:102F8000300A000000000000417373657274696FBD
:102F90006E206661696C65643A2074662D3E6570CA
:102FA0006320252034203D3D20300A000000000031
:102FB000417373657274696F6E206661696C6564D4
:102FC0003A202122756E65787065637465642065AA
:102FD0007863657074696F6E220A0000000000005B
:102FE000417373657274696F6E206661696C6564A4
:102FF0003A202122756E737570706F72746564204B
:0C30000073617470206D6F6465220A001B
:10400000EFBEEFBEEFBEEFBEEFBEEFBEEFBEEFBE48
:04401000EFBEEFBE52
:040000058000000077
:00000001FF
